:041800000CEF0CF0ED
:10180800FACF2BF0FBCF2CF0E9CF2DF097ED18F0A5
:0C181800EFEF1AF08C0F8C0F020104FCA3
:021826001500AB
:10251F000102FC030328C408F51200A6A21200FD55
:10252F00D7010ECBEC1EF01200020ECBEC1EF012F8
:10253F0000020E9AEC1FF01200D6CF03F0D7CF0493
:10254F00F003C001F004C002F0120001C0A9FFA601
:10255F009CA69EA68000F000F0A8501200D6CF6275
:10256F00F0D7CF63F062C060F063C061F01200601B
:10257F00C0A9FFA69CA69EA68000F000F0A850124E
:10258F00000001606F010E0001F06F60C0EFF002FC
:10259F000100511200016E01507F0BD56E000ED756
:1025AF006E000ED66EF29401AE02D0F28A01D0F216
:1025BF009AD58E1200000E026E000E016EADEC1257
:1025CF00F00001E26F040E0001E26503D0000E007F
:1025DF0001E26F12000001E251050D550EF32400C8
:1025EF0001616F7F0EF4200001626F050E00016321
:1025FF006F44EC17F012000001E651040D820EF348
:10260F00240001616F7F0EF4200001626F040E0041
:10261F0001636F44EC17F012000001E851050D96AD
:10262F000EF3240001616F7F0EF4200001626F052D
:10263F000E0001636F44EC17F012000001EC51061D
:10264F000DB30EF3240001616F7E0EF420000162C2
:10265F006F060E0001636F44EC17F012000001E1EA
:10266F0051040D1F0EF3240001616F7F0EF4200043
:10267F0001626F040E0001636F44EC17F01200004B
:10268F0001EB51060DD70EF3240001616F7E0EF49E
:10269F00200001626F060E0001636F44EC17F01209
:1026AF00000001F151050DF90EF3240001616F7D5A
:1026BF000EF4200001626F050E0001636F44EC17EA
:1026CF00F012000001F351040DC80EF32400016154
:1026DF006F7F0EF4200001626F040E0001636F44E0
:1026EF00EC17F01200000E0001616F000E00016088
:1026FF006FBFEC12F00001E26F040E0001E2650300
:10270F00D0000E0001E26F1200010E0001606F0099
:10271F0001E251030AD8B408D00001E251040AD8EB
:10272F00B403D0000E0001606F0001605112006908
:10273F008468986D82010E0001E46F000E166E75AD
:10274F000E156E000E186E000E176E000E1A6E002C
:10275F000E196E61EC18F012000001EF510001F03C
:10276F005DD8A002D0000E0CD00001F051010D0277
:10277F0001000EF324D96E0201020EF420DA6EDF8F
:10278F0050120002C008F001C007F008D007C0D9EE
:10279F00FF08C0DAFF03C0DFFF074A082A0506D883
:1027AF00A006060528D8B40628D8B41200EFD7041F
:1027BF0001040E0001D16F0401280E0001D06F003B
:1027CF000E0001D56F080E0001D46F250E0001D742
:1027DF006F240E0001D66F0001D38F12000001E2AB
:1027EF002B040E0001E26503D0000E0001E26F958D
:1027FF00EC12F0000E0001616F000E0001606FE23D
:10280F00C062F095EC15F0F2EC12F012000001E648
:10281F002B040E0001E66503D0000E0001E66F9554
:10282F00EC12F0000E0001616F030E0001606FE605
:10283F00C062F095EC15F003EC13F012000001E804
:10284F002B030E0001E86503D0000E0001E86F9521
:10285F00EC12F0000E0001616F060E0001606FE8D0
:10286F00C062F095EC15F014EC13F012000001ECBF
:10287F002B050E0001EC6503D0000E0001EC6F95E7
:10288F00EC12F0000E0001616F010E0001606FECA1
:10289F00C062F095EC15F025EC13F012000001E189
:1028AF002B060E0001E16503D0000E0001E16F95CC
:1028BF00EC12F0000E0001616F050E0001606FE178
:1028CF00C062F095EC15F036EC13F012000001EB3E
:1028DF002B050E0001EB6503D0000E0001EB6F9589
:1028EF00EC12F0000E0001616F040E0001606FEB3F
:1028FF00C062F095EC15F047EC13F012000001F1F7
:10290F002B070E0001F16503D0000E0001F16F954A
:10291F00EC12F0000E0001616F020E0001606FF10A
:10292F00C062F095EC15F058EC13F012000001F3B3
:10293F002B020E0001F36503D0000E0001F36F951B
:10294F00EC12F0000E0001616F080E0001606FF3D2
:10295F00C062F095EC15F069EC13F012000001E580
:10296F006715D0000E6D6E000E696E160E6F6E9F9E
:10297F000E6B6E7B0E696ED08EA28AA08AF28E01CC
:10298F00D06D866DA6FDD7010E0001E56F12000018
:10299F000161516011D8A402D0270E12D00001613D
:1029AF00516011D8B40CD00A0E0001605D000E000A
:1029BF00016159D8B004D0000160511D0F01D02C16
:1029CF000E12000001685100016A03F3CF6CF0F49E
:1029DF00CF6DF00001685100016B03F35000016DE2
:1029EF00270001695100016A03F35000016D276C44
:1029FF00C068F06DC069F01200000E0001E46F00B6
:102A0F000E166E740E156E000E186E000E176E00F9
:102A1F000E1A6E000E196E61EC18F06D92699468C3
:102A2F00B869A803D0689801D0689468A41200FC14
:102A3F00D7000161C067F0000160C066F00AD06680
:102A4F00C0D9FF67C0DAFF000162C0DFFF00016677
:102A5F004B672B00016407D8A0650700016429D8D4
:102A6F00B46529D8B41200EBD70001646FFE0EF6DF
:102A7F006E170EF76E0900F5CF62F00900F5CF6300
:102A8F00F0020E0001625D000E6359D8A005D00060
:102A9F000164519DEC17F004D000016451F5EC1561
:102AAF00F012000001646FFE0EF66E170EF76E093E
:102ABF0000F5CF62F00900F5CF63F0020E0001625E
:102ACF005D000E6359D8A005D000016451F5EC15D7
:102ADF00F004D0000164519DEC17F0120070A01BA0
:102AEF00D0800E3DC0D9FF3EC0DAFFDF6213D08425
:102AFF000ED8C0D9FFD9C0DAFFDF620CD03DC0D9E4
:102B0F00FF3EC0DAFF0C0EDF6E3DC0D9FF3EC0DACC
:102B1F00FF000EDB8E7090689A1200000E000163AA
:102B2F006F60C0A9FF62C0A8FFA69EA69CA68400E6
:102B3F000EF2BE010E0001636FF29E550EA76EAA34
:102B4F000EA76EA682A6B2FED7000163B102D0F225
:102B5F009E01D0F28EA69412006DA217D0010E3CEA
:102B6F00EC15F0020E3CEC15F0030E3CEC15F013D7
:102B7F00D081EC16F010D0010E59EC15F0020E5961
:102B8F00EC15F0030E59EC15F006D00001E55120BD
:102B9F000AD8B4EED7F0D71200000E9AEC1FF0F35C
:102BAF00EC16F0DDEC29F0B6EC14F0B4EC15F020D7
:102BBF000E0001E55DD8A0F9D76DA208D056EC1A2A
:102BCF00F00009D8B4F2D717EC16F0EFD70001E4F4
:102BDF0051D8A4EBD754EC33F0E8D70001606F1352
:102BEF00D058C0D9FF59C0DAFF5C500BD05AC0D9AA
:102BFF00FF5BC0DAFF5D5005D094C1D9FF95C1DAF4
:102C0F00FF5E50DF120BD000016051010AD8B4E80B
:102C1F00D7030AD8B4EBD7010AD8B4EED712000005
:102C2F0001E351D8B41DD00001E451D8B419D0A09C
:102C3F009AA0EC12F06D92180E00016B6F5F0EE808
:102C4F002EFED76B2FFCD700F06D84100E00016B9A
:102C5F006F940EE82EFED76B2FFCD700D06D94A08B
:102C6F008A12000E6E09A405D0000E016E0E50A23E
:102C7F00EC1AF009A205D0010E016E0E50A2EC1A4B
:102C8F00F00E50010D700E0A6E0F0E0B6EF3500A00
:102C9F0026F4500B220AC00CF00BC00DF00CC0D95B
:102CAF00FF0DC0DAFF09C0DFFF12000001EF510076
:102CBF0001F05DD8A005D0000E0001F06F000E18D6
:102CCF00D00001F051010D0201000EF324D96E0264
:102CDF0001020EF420DA6EDF500001606F0001F088
:102CEF002B0001606703D0000E0001F06F00016040
:102CFF0051120005010851CCEC16F00001666F006F
:102D0F000166A104D0010E59EC15F003D0010E3C61
:102D1F00EC15F0000166A304D0020E59EC15F00378
:102D2F00D0020E3CEC15F0000166A504D0030E593D
:102D3F00EC15F003D0030E3CEC15F01200000E0062
:102D4F0001656F000106D0000166511AEC17F00003
:102D5F0001652B00016551010D000161C063F00099
:102D6F000162C064F0F35000016327F45000016466
:102D7F002363C0F6FF64C0F7FF08000001F5CF66BC
:102D8F00F000016667E0D712000001656F65C0EAC9
:102D9F00F00001655168EC1EF00001656FFE0EF644
:102DAF006E170EF76E0900F5CF63F00900F5CF64CB
:102DBF00F0030E0001635D000E6459D8B009D04FC7
:102DCF002A030E4F6403D0000E4F6E02D000016530
:102DDF0093000165511200FE0EF66E170EF76E0985
:102DEF0000F5CF65F00900F5CF66F0030E00016521
:102DFF005D000E6659D8A00CD00F0E5B6E8B0E5A6D
:102E0F006E5BC059F05AC058F0010E5C6E020E5D39
:102E1F006E010E59EC15F0020E59EC15F0030E5918
:102E2F00EC15F012000001606F800E0001F05DD80C
:102E3F00B010D00001F051010D0201000EF324D9A2
:102E4F006E0201020EF420DA6E000160C0DFFF0097
:102E5F0001F02B800E0001F05DD8B00DD00001F015
:102E6F0051010D0201000EF324D96E0201020EF47E
:102E7F0020DA6E000EDF6E1200000E0001676F0089
:102E8F000106D0000166511AEC17F00001672B0004
:102E9F00016751010D000161C064F0000162C0655E
:102EAF00F0F35000016427F4500001652364C0F66D
:102EBF00FF65C0F7FF08000001F5CF66F000016362
:102ECF00510001675DD8B003D000016667DAD712F1
:102EDF00004950020AD8A403D060EC27F025D00097
:102EEF000E496E42661FD020EE01F03F50D92640AA
:102EFF0050DA22080EDF6E20EE02F03F50D9264046
:102F0F0050DA22200EDE6E040EDD6E3FC0D9FF4078
:102F1F00C0DAFF0C0EDF6E3FC0D9FF40C0DAFF00F2
:102F2F000EDB8E02D0000E426E12000001616F1E8A
:102F3F00D05C50FF0A0001606F58C0D9FF59C0DA4A
:102F4F00FF11D05D50FF0A0001606F5AC0D9FF5BBF
:102F5F00C0DAFF08D05E50FF0A0001606F94C1D93C
:102F6F00FF95C1DAFF00016051DF160BD000016140
:102F7F0051010AD8B4DDD7030AD8B4E3D7010AD870
:102F8F00B4E9D71200000E026E010E016EADEC1205
:102F9F00F00001EC6F050E0001EC6503D0000E0090
:102FAF0001EC6F000E026E050E016EADEC12F0001B
:102FBF0001E16F060E0001E16503D0040E0001E18F
:102FCF006F000E026E060E016EADEC12F00001E8FE
:102FDF006F030E0001E86503D0000E0001E86F12C9
:102FEF0000000E0001616F010E0001606FBFEC1257
:102FFF00F00001EC6F050E0001EC6503D0000E0030
:10300F0001EC6F000E0001616F050E0001606FBFD4
:10301F00EC12F00001E16F060E0001E16503D00430
:10302F000E0001E16F000E0001616F060E000160DE
:10303F006FBFEC12F00001E86F030E0001E86503AB
:10304F00D0000E0001E86F1200000171C077F00090
:10305F000170C076F000016FC075F000016EC07492
:10306F00F01DD0000176C0F6FF000177C0F7FFF822
:10307F006A74C0D9FF75C0DAFF070EF76403D00872
:10308F0000F55005D0F6CFE1FFF7CFE2FFE750DFB5
:10309F006E0001764B772B0001744B752B0001727C
:1030AF0007D8A0730700017229D8B47329D8B412B6
:1030BF0000D8D70CD098EC12F031D09CEC12F02E37
:1030CF00D081EC2BF02BD025EC25F028D015C01B90
:1030DF00F016C01CF01C50000AD8B404D07F0AD8D8
:1030EF00B41BD01CD01B50010AD8B4EAD7030AD89E
:1030FF00B415D0010AD8B4E7D7060AD8B40FD077E1
:10310F000AD8B40CD0010AD8B409D0070AD8B4D55C
:10311F00D7010AD8B4CFD702D01B50FF0A1200062E
:10312F0000EACF2EF0E1CF2FF0E2CF30F0D9CF3140
:10313F00F0DACF32F0F3CF33F0F4CF34F0F6CF35FF
:10314F00F0F7CF36F0F8CF37F0F5CF38F030EC2678
:10315F00F038C0F5FF37C0F8FF36C0F7FF35C0F6BF
:10316F00FF34C0F4FF33C0F3FF32C0DAFF31C0D9F0
:10317F00FF30C0E2FF2FC0E1FF2EC0EAFF2DC0E9F4
:10318F00FF2CC0FBFF2BC0FAFF1100000161C067CD
:10319F00F0000160C066F020D0000166C0F6FF00AD
:1031AF000167C0F7FFF86A070EF76403D00800F550
:1031BF005005D0F6CFE1FFF7CFE2FFE750000162F5
:1031CF0019D8A407D0000167C061F0000166C06084
:1031DF00F013D00001664B672B00016407D8A06580
:1031EF000700016429D8B46529D8A4D6D7000E00EA
:1031FF0001616F000E0001606F1200000E0001638D
:10320F006F0001E951D8B42FD060C0D9FF61C0DA87
:10321F00FFDF500001626FDD0E00016217D8A4239B
:10322F00D0000120EE01F000016051D926000161AC
:10323F0051DA22DF500001626F000162B114D00039
:10324F0001EC51D8B410D04A50D8B40AD00001F1D3
:10325F0051040AD8B408D00001F151050AD8B403BB
:10326F00D0010E0001636F00016351120000016B6A
:10327F006F27D0010E0001E96F31D0000E0001E978
:10328F006F000E0001F26F2AD000016951D8B426E9
:10329F00D08CEC13F00009D8B421D0010E4A1A1EBD
:1032AF00D068C06AF0220E00016A17D8B417D08C0C
:1032BF00EC13F00009D8B412D0870E00016B6F0E1B
:1032CF00D000016B51270AD8B4EBD71E0AD8B4DC53
:1032DF00D7A90AD8B4CED7010AD8B4CFD700016B7B
:1032EF0051120036D062C0D9FF63C0DAFFDF500041
:1032FF0001666F60C0D9FF61C0DAFFDF5000016661
:10330F0019D8B420D062C0D9FF63C0DAFFDF5000F4
:10331F0001666F676B0001661F671F664B672B6047
:10332F00C0D9FF61C0DAFFDF500001686F0001688C
:10333F0051000166250001606F000E00016721003A
:10334F0001616F16D00001604B612B0001624B636E
:10335F002B00016407D8A0650700016429D8B46564
:10336F0029D8A4C0D7000E0001616F000E000160C4
:10337F006F1200000E4E6E000E456E000E436E0073
:10338F000E446E000E426E000E496ED8C0D9FFD9A2
:10339F00C0DAFF7F0EDF16040E0001D81BD8C0D98C
:1033AF00FFD9C0DAFF7F0EDF16040E0001D81B3FD6
:1033BF00C0D9FF40C0DAFF7F0EDF16000E0001F804
:1033CF006F000E0001FA6F000E0001F96F000E0082
:1033DF0001D36F000E0001D56F000E0001D46F56A0
:1033EF00EC21F0000E166E030E156E000E186E0017
:1033FF000E176E000E1A6E000E196E61EC18F0CEDD
:10340F00EC21F012000001646F7D0E0001636F7CF0
:10341F000E0001626F000E0001656F39D00001656B
:10342F0051010D000162C060F0000163C061F0F353
:10343F005000016027F4500001612360C0F6FF6166
:10344F00C0F7FF0800F55000016419D8A41ED00082
:10345F0001EB51070D7C0E0001606F7D0E616FF364
:10346F005000016027F450000161230001655101F4
:10347F000DF35000016027F4500001612360C0F686
:10348F00FF61C0F7FF0800F55008D00001652B065B
:10349F000E00016565C3D7000164511200FE0EF6E0
:1034AF006E170EF76E0900F5CF60F00900F5CF61CA
:1034BF00F0030E0001605D000E6159D8A006D00127
:1034CF000E0001F46F070E0001FF6FFE0EF66E1770
:1034DF000EF76E0900F5CF60F00900F5CF61F0042B
:1034EF000E0001605D000E6159D8A002D0F30E5F8F
:1034FF006EF4C092FF000E966E010E0001636F8393
:10350F0050FF0A5F140009D8A40CD08150FF0A00A5
:10351F0001606F3F0E00016017D8A403D0000E00AA
:10352F0001636F63C062F03F0E926EFFC096FF00A3
:10353F000162511200066E0401040E086E040100B0
:10354F000E076E0150026E036AD8900236033606DC
:10355F0050046E056AD89004360536D890043605A7
:10356F00360250042603500522D89004360536D86B
:10357F009004360536045007260550082207C0D997
:10358F00FF08C0DAFFDF9E016607D00650020D3933
:10359F000EF324D96E000E08D00650020D0001D88C
:1035AF000EF324D96E0001000EF420DA6E07C0DE90
:1035BF00FF08C0DDFF07C0D9FF08C0DAFFDF9C207E
:1035CF00EE04F00750D9260850DA22DF8C120002E1
:1035DF00EE00F0800EEE6AE806FDE101EE9EF0458A
:1035EF000EEE6AE806FDE100EED0F02B0EEE6AE873
:1035FF0006FDE100EE39F01F0EEE6AE806FDE1165A
:10360F000EF66E370EF76E000EF86E01EE00F0102C
:10361F00EE9EF00900F5CFEEFFE550E150FAE11F05
:10362F000EF66E250EF76E000EF86E00EEFBF01024
:10363F00EE05F00900F5CFEEFFE550E150FAE11C81
:10364F000EF66E180EF76E000EF86E00EE58F010B4
:10365F00EE08F00900F5CFEEFFE550E150FAE1007A
:10366F000EF86E0001D4EF15F0000E436E000E44FD
:10367F006E4950020AD8A41DD020EE01F03F50D958
:10368F00264050DA22080EDF6E20EE02F03F50D9AE
:10369F00264050DA22280EDE6E040EDD6E3FC0D9B2
:1036AF00FF40C0DAFF480EDF6E3FC0D9FF40C0DADF
:1036BF00FF27D00001F9510401265D0001FA5104E2
:1036CF00012759D8B004D026C4F9F027C4FAF0E284
:1036DF00EC20F0000120EE02F00001D851D92600B5
:1036EF0001D951DA22280EDE6E040EDD6ED8C0D954
:1036FF00FFD9C0DAFF480EDF6ED8C0D9FFD9C0DAC4
:10370F00FF000EDB8E1200830F830F830F830F8357
:10371F000F830F810F810F810F810F810F810F8118
:10372F000F810F810F810F810F810F830F830F8304
:10373F000F830F830F830F920F920F920F920F929F
:10374F000F920F960F960F960F960F960F920F924E
:10375F000F920F920F920F1020408004082010023A
:10376F000104088040201008042010080401020101
:10377F00020408102080402010020100000E0E0EDF
:10378F000E0E0E0102040810200102020408102080
:10379F0001020404020120100804028B0F00000E26
:1037AF000E0E0E0E0E0101010E026E0101A60E018C
:1037BF006E000E046E0E0E036E000E066E1E0E05CC
:1037CF006EC9EC13F0000E026E020E016EADEC121C
:1037DF00F00001F16F070E0001F16503D0000E003C
:1037EF0001F16F000E026E040E016EADEC12F000CF
:1037FF0001EB6F050E0001EB6503D0000E0001EB2E
:10380F006F000E026E030E016EADEC12F00001E6BA
:10381F006F040E0001E66503D0000E0001E66F0095
:10382F000E026E080E016EADEC12F00001F36F0187
:10383F000E0001F36503D0000E0001F36FE2EC12EE
:10384F00F0CAEC17F012000001706F000170C06039
:10385F00F00001616B000E0001636F0C0E0001623E
:10386F006F06EC1EF0000160510001716F0001EA5C
:10387F00A13FD0060E000171653BD0070E0001710C
:10388F005F000E0001636F0C0E0001626F0001708C
:10389F00C060F00001616B71EC20F0000160C06846
:1038AF00F0000161C069F0000E00016B6F050E00A2
:1038BF00016A6FE9EC14F04F0E00016E6F770E6F17
:1038CF006F0001685100016E270001695100016FFF
:1038DF002300017151010DF35000016E27F45000C8
:1038EF00016F236EC0F6FF6FC0F7FF0800F55001A0
:1038FF00D0000E12000101010E0001616F0101A63F
:10390F000E0001606F000E0001636F0E0E0001626A
:10391F006F000E0001656F1E0E0001646F20EC1525
:10392F00F0000E0001616F020E0001606FBFEC121C
:10393F00F00001F16F070E0001F16503D0000E00DA
:10394F0001F16F000E0001616F040E0001606FBF87
:10395F00EC12F00001EB6F050E0001EB6503D000D8
:10396F000E0001EB6F000E0001616F030E0001608E
:10397F006FBFEC12F00001E66F040E0001E6650365
:10398F00D0000E0001E66F000E0001616F080E00FF
:10399F0001606FBFEC12F00001F36F010E0001F335
:1039AF006503D0000E0001F36F7AEC13F0F8EC17FB
:1039BF00F01200056E0150D8B409D00550020D0069
:1039CF0001D80EF324D96E0001000E06D005500267
:1039DF000D390EF324D96E000EF420DA6EDECF0609
:1039EF00F0DDCF07F007500610D8A405D0000E0267
:1039FF006E000E016E3ED020EE02F00650D9260763
:103A0F0050DA2202C0DEFF03C0DDFF20EE01F00618
:103A1F0050D9260750DA2204C0DFFF06C0D9FF07AE
:103A2F00C0DAFF400EDF1606C0D9FF07C0DAFF006D
:103A3F000EDB8606C0D9FF07C0DAFF000EDB8E0152
:103A4F0050D8B409D00550020D0001D80EF324D977
:103A5F006E0001000E06D00550020D390EF324D969
:103A6F006E000EF420DA6E040EDF1A07C002F006A5
:103A7F00C001F0120046665FD0010E466E47665BCE
:103A8F00D0010E476E4950020AD8A418D000012069
:103A9F00EE01F00001D851D9260001D951DA2200E8
:103AAF000EDF6ED8C0D9FFD9C0DAFF480EDF6ED84F
:103ABF00C0D9FFD9C0DAFF000EDB8E3DD04904D844
:103ACF00A43AD0000E426E20EE01F03D50D9263EB2
:103ADF0050DA22080EDF6E20EE02F03D50D9263E5E
:103AEF0050DA22200EDE6E040EDD6E3DC0D9FF3E91
:103AFF00C0DAFF040EDF6E3DC0D9FF3EC0DAFF0013
:103B0F000EDB8E010E426E20EE01F03F50D92640A3
:103B1F0050DA22080EDF6E20EE02F03F50D9264019
:103B2F0050DA22200EDE6E040EDD6E3FC0D9FF404C
:103B3F00C0DAFF800EDF6E1200000E0401286F0046
:103B4F000E0401296F3ED00001F88F0001E305D864
:103B5F00A444D00401288341D00001F88F3ED00047
:103B6F0001F88F040124BF0BD0040124510F0B0166
:103B7F006E0150020D390EF324D96E000E0CD004D5
:103B8F000124510F0B016E0150020D0001D80EF3ED
:103B9F0024D96E0001000EF420DA6EDECF02F0DDC4
:103BAF00CF03F002C0D9FF03C0DAFFDFAE16D00299
:103BBF00C0D9FF03C0DAFFDFA410D0010E04012823
:103BCF006F0CD0040120511F0B000AD8B4BCD701D1
:103BDF000AD8B4C2D7030AD8B4C2D70001F8AF0DC0
:103BEF00D00401040E0001F66F0401280E0001F548
:103BFF006F0001F881020E0001F96F1200000E0034
:103C0F0001656F00016151800AF36E800EF35C0055
:103C1F000ED8B4605DD8B009D00001606D000161AD
:103C2F001FD8B0612B010E0001656F000163518039
:103C3F000AF36E800EF35C000ED8B4625DD8B00646
:103C4F00D00001626D0001631FD8B0632B000163C8
:103C5F00516211D8B426D0010E0001646F06D00056
:103C6F0001D890623763370001642B000163AFF70F
:103C7F00D7000162510001605D00016351000161D5
:103C8F0059D8A008D0000162510001605F000163A4
:103C9F00510001615B0001D890633362330001640E
:103CAF002FE7D700016551D8B406D00001606D0031
:103CBF0001611FD8B0612B60C060F061C061F0126C
:103CCF00000001626F0001EC51D8A437D059D0E148
:103CDF00C060F0010E0001616F0001602B03D00086
:103CEF0001D89061370001602FFAD700016151FFB1
:103CFF000A00016217E1C060F0E9C061F0000160E5
:103D0F002B03D00001D89061370001602FFAD71034
:103D1F00D0E1C060F0FD0E00016027E9C061F00046
:103D2F0001602B03D00001D89061370001602FFA9A
:103D3F00D7000161510001621314D00001E151005D
:103D4F000AD8B4C5D7010AD8B4C2D7030AD8B4BFAA
:103D5F00D7010AD8B4DDD7070AD8B4DAD7010AD801
:103D6F00B4D7D70001F351020AD8A40AD00001F248
:103D7F00A302D0000162810001F2AB02D000016208
:103D8F00850001625112000B6E59D0000EBD6E00FE
:103D9F000EBA6E0F0EC16EFE0EF66E170EF76E098F
:103DAF0000F5CF09F00900F5CF0AF0030E095C000A
:103DBF000E0A58D8A01DD0000EC26E0E0EC16E9EF8
:103DCF000EC06EFE0EF66E170EF76E0900F5CF09D8
:103DDF00F00900F5CF0AF00950030A0A10D8A4021F
:103DEF00D0FE0E01D0F30E0001FD6F070E0001FE95
:103DFF006F000E896E3F0E926E000E8A6E9368F101
:103E0F009E000E8B6E380E946E000E8C6EFDC0955C
:103E1F00FF848E000E8D6EFEC096FFDAEC1BF0183D
:103E2F00D0130ED36E15D0600ED36E100E096E9494
:103E3F000EE82EFED7092EFCD700D00AD00B50006B
:103E4F000AD8B4A3D7010AD8B4EBD7030AD8B4EB76
:103E5F00D71200D8C0D9FFD9C0DAFF000EDFBC01DE
:103E6F000E026E040E0001D81B0001E551080AD89E
:103E7F00A40CD0040122517F0B6E6E6E50D8B40289
:103E8F00D0100E01D0040E0001E56F4904D8A42E06
:103E9F00D0000120EE02F00001D851D9260001D93F
:103EAF0051DA22280EDE6E040EDD6EE2EC20F04EAB
:103EBF0050020AD8A406D0D8C0D9FFD9C0DAFF045F
:103ECF000E0DD0026606D0D8C0D9FFD9C0DAFF4890
:103EDF000E05D0D8C0D9FFD9C0DAFF080EDF6ED8D3
:103EEF00C0D9FFD9C0DAFF000EDB8E1BD00001D383
:103EFF00AF16D00001D751D611D8B40FD000012082
:103F0F00EED6F001D80AD00500FA6EDE50FD6EDE57
:103F1F0050FE6EF850FF6EFA5012000001D39F0052
:103F2F000E496E120000016A6F5CD0000EBD6E006C
:103F3F000EBA6E0F0EC16EFE0EF66E170EF76E09ED
:103F4F0000F5CF68F00900F5CF69F0030E000168A6
:103F5F005D000E6959D8A01ED0000EC26E0E0EC1A4
:103F6F006E9E0EC06EFE0EF66E170EF76E0900F502
:103F7F00CF68F00900F5CF69F000016851030A69B5
:103F8F0011D8A402D0FE0E01D0F30E0001FD6F0771
:103F9F000E0001FE6F000E896E3F0E926E000E8AAC
:103FAF006E9368F19E000E8B6E380E946E000E8C21
:103FBF006EFDC095FF848E000E8D6EFEC096FF8243
:103FCF00EC1CF01AD0130ED36E17D0600ED36E10F8
:103FDF000E0001686F940EE82EFED7682FFCD700F5
:103FEF00D00BD000016A51000AD8B49FD7010AD86C
:103FFF00B4E9D7030AD8B4E9D712002D0E486E558D
:10400F00C027F0FD0E2716D8A45AD055C027F0D8D8
:10401F009027323F0E27162750040D0401000EF390
:10402F00243D6E0401040EF4203E6E3EC040F03D70
:10403F00C03FF0040E3F1A3DC0D9FF3EC0DAFFDF8C
:10404F0030E8320F0B0D0AD8A437D0000E296E249A
:10405F00D020EE02F03D50D9263E50DA22DECF2797
:10406F00F0DDCF28F027C0D9FF28C0DAFF29500193
:10407F000D0401200EF324E16E0401040EF420E27E
:10408F006EDFCFE7FF20EE02F03D50D9263E50DA2B
:10409F0022DE2A000EDD22292A070E2964D9D72015
:1040AF00EE02F03D50D9263E50DA22200EDE6E048D
:1040BF000EDD6EC1EC19F00CD070EC17F009D05575
:1040CF00C027F0FD0E27162750040AD8B431EC1F75
:1040DF00F01200000E0001656F00016351800AF3BA
:1040EF006E800EF35C000ED8B4625DD8B009D000BC
:1040FF0001626D0001631FD8B0632B010E000165D3
:10410F006F00016151800AF36E800EF35C000ED8D0
:10411F00B4605DD8B009D00001606D0001611FD897
:10412F00B0612B010E0001651B000E0001676F00CF
:10413F000E0001666F000163516211D8B42CD001DB
:10414F000E0001646F06D00001D89062376337000C
:10415F0001642B000163AFF7D70001D89066376772
:10416F0037000162510001605D0001635100016180
:10417F0059D8A00AD0000162510001605F000163AD
:10418F00510001615B000166810001D890633362C9
:10419F00330001642FE1D700016551D8B406D00078
:1041AF0001666D0001671FD8B0672B66C060F067AE
:1041BF00C061F01200080E016E080E0001F95D00DB
:1041CF000E0001FA59D8B00BD0F9C001F04E6602BB
:1041DF00D0010E04D04E04D8A402D0020E4E6E01B0
:1041EF00500001F95F000E0001FA5B000120EE01A3
:1041FF00F00001D851D9260001D951DA2201C0DFD0
:10420F00FF0401040E0101A36F0401280E0101A296
:10421F006F0001F8A11FD03FD00001F5C0F6FF00DD
:10422F0001F6C0F7FFF86AA2C1D9FFA3C1DAFF07F1
:10423F000EF76403D00800F55005D0F6CFE1FFF775
:10424F00CFE2FFE750DF6E0001F54BF62B0101A225
:10425F004BA32B01060166E0D720D00001F5C0F675
:10426F00FF0001F6C0F7FFF86AA2C1D9FFA3C1DAB8
:10427F00FF070EF76403D00800F55005D0F6CFE125
:10428F00FFF7CFE2FFE750DF6E0001F54BF62B0192
:10429F0001A24BA32B01060166E0D71200040120F7
:1042AF0039E832030B0009D8A470D04ED00001F8C2
:1042BF008F080E0001E56F69D097EC28F066D0BE2D
:1042CF00EC22F063D0000E0001F66F530E0001F5E3
:1042DF006F15D0A4EC1DF059D089EC2CF056D004FA
:1042EF00012451010D540E256E000E266EF350253C
:1042FF0026F450262225C0F5F026C0F6F00001F86E
:10430F0081010E0001F96F0001F88F3FD00001F815
:10431F008F04012451010D540EF324D96E000EF4B5
:10432F0020DA6E040122C4DFFF30D0000E166E02B9
:10433F000E156E000E186E000E176E000E1A6E0020
:10434F000E196E61EC18F021D004012151000AD82A
:10435F00B4C0D7010AD8B4C0D7020AD8B4BDD706A3
:10436F000AD8B4A4D7030AD8B4A7D7010AD8B4DDA2
:10437F00D70F0AD8B4A7D7010AD8B4A1D7030AD840
:10438F00B4AED7010AD8B4C2D7070A12006D98008D
:10439F0001F8BF39D00001D3AF0BD0020E496E44E4
:1043AF006602D03CEC1BF0000E476E000E466E65A9
:1043BF00D020EE01F03F50D9264050DA22080EDF10
:1043CF006E20EE02F03F50D9264050DA22200EDE4A
:1043DF006E040EDD6E3FC0D9FF40C0DAFF0C0EDF5A
:1043EF006E3FC0D9FF40C0DAFF000EDB8ED8C0D9B8
:1043FF00FFD9C0DAFF040EDF6ED8C0D9FFD9C0DAFB
:10440F00FF000EDB8E3AD0040120AF0FD0010E4912
:10441F006E436602D03CEC1BF0000E476E000E465A
:10442F006E45662BD042EC1DF028D0020E496E204F
:10443F00EE01F03F50D9264050DA22080EDF6E20F1
:10444F00EE02F03F50D9264050DA22200EDE6E04E5
:10445F000EDD6E3FC0D9FF40C0DAFF040EDF6E3FA6
:10446F00C0D9FF40C0DAFF000EDB8E000E476E0092
:10447F000E466E456602D042EC1DF012000001643C
:10448F006F00016051D8B40AD000016451020D00D1
:10449F0001D80EF324D96E0001000E07D00001647D
:1044AF0051020D390EF324D96E000EF420DA6E008E
:1044BF0001DECF65F00001DDCF66F00001665165CA
:1044CF0011D8A407D0000E0001616F000E0001602B
:1044DF006F4CD0000120EE02F000016551D926008B
:1044EF00016651DA22000161C0DEFF000162C0DD0A
:1044FF00FF000120EE01F000016551D92600016691
:10450F0051DA22000163C0DFFF65C0D9FF66C0DA50
:10451F00FF400EDF1665C0D9FF66C0DAFF000EDB65
:10452F008665C0D9FF66C0DAFF000EDB8E00016022
:10453F0051D8B40AD000016451020D0001D80EF316
:10454F0024D96E0001000E07D000016451020D390D
:10455F000EF324D96E000EF420DA6E040EDF1A006B
:10456F000166C061F0000165C060F012000001F843
:10457F008F0F0E026E710E016E000E046E000E0391
:10458F006E000E066E010E056EC9EC13F0040104E9
:10459F000E026E0401000E016E000E046E000E037B
:1045AF006E000E066E200E056EC9EC13F06D8C00BA
:1045BF000E1D6E19D01D50010D0001DC0EF324D914
:1045CF006E0001000EF420DA6E000EDF6E1D50013A
:1045DF000D0001DE0EF324D96E0001000EF420DA77
:1045EF006E000EDF6E1D2A010E1D64E4D7000E0251
:1045FF006E540E016E000E046E000E036E000E065A
:10460F006E010E056EC9EC13F06D9C0401040E00D3
:10461F0001D96F0401080E0001D86F0401040E3E8A
:10462F006E0401000E3D6E3EC040F03DC03FF022D3
:10463F00C453F0536602D0100E0FD0000E166E0149
:10464F000E156E000E186E530E176E000E1A6E01B9
:10465F000E196E61EC18F0200E0001E56F120000CC
:10466F000E0001696F000E00016A6F000E00016CF1
:10467F006F12D000016C51010D0101D80EF324D936
:10468F006E0101010EF420DA6E010EDF6402D0001C
:10469F0001692B00016C2B070E00016C65EAD70036
:1046AF000E00016C6F12D000016C51010D0101C49D
:1046BF000EF324D96E0101010EF420DA6E010EDF24
:1046CF006402D000016A2B00016C2B0B0E00016CF1
:1046DF0065EAD7000E00016B6F010E0001696507D7
:1046EF00D0010E00016A6503D0010E00016B6F6BE4
:1046FF00C068F00101010E0001616F0101D80E00C9
:10470F0001606F000E0001636F000E0001626F0009
:10471F000E0001656F080E0001646F20EC15F001AB
:10472F0001010E0001616F0101C40E0001606F00F5
:10473F000E0001636F000E0001626F000E00016535
:10474F006F0C0E0001646F20EC15F0000168511220
:10475F0000000163C06BF0000162C06AF0000161EC
:10476F00C069F0000160C068F00001685100016A83
:10477F005D0001695100016B59D8B044D000016A46
:10478F00C066F000016BC067F00001645100016664
:10479F002700016551000167230001665100016880
:1047AF005D0001675100016959D8B02CD000016438
:1047BF005100016A270001655100016B230001645C
:1047CF005100016827000165510001692300016A4A
:1047DF0007D8A06B076AC0D9FF6BC0DAFF0001686A
:1047EF0007D8A0690768C0E1FF69C0E2FFDFCFE724
:1047FF00FF00016407D8A06507000165516411D857
:10480F00B41FD0E4D7000165516411D8B419D06A30
:10481F00C0D9FF6BC0DAFF68C0E1FF69C0E2FFDFFC
:10482F00CFE7FF00016A4B6B2B0001684B692B0030
:10483F00016407D8A06507000165516411D8A4E78A
:10484F00D71200020E0001806F78C0D9FF79C0DA4D
:10485F00FFDF5000017E6F020E0001816F62D000FA
:10486F00018151010DF35000017825D96EF45000EC
:10487F00017921DA6EDF5000017F6F00017F512B2C
:10488F00EC1CF00001826F0001826706D000017FEF
:10489F0051A8EC25F00001826F00018251D8B43F7E
:1048AF00D0080E0001805DD8B03AD07EC068F0020B
:1048BF000E00017A250001606F000E00017B2100C0
:1048CF0001616F000182C062F00001636B000E0096
:1048DF0001656F060E0001646FCDEC18F0000161E9
:1048EF005100016011D8A402D0010E01D0000E00BA
:1048FF0001696F000182513EEC19F00001826F00D7
:10490F00018051010DF35000017C25D96EF4500048
:10491F00017D21DA6E000182C0DFFF0001802B00D4
:10492F0001812B070E000181659AD77CC0D9FF7DCD
:10493F00C0DAFF00017EC0DFFF010E12000001721E
:10494F006F0001F151040AD8B405D00001F15105EF
:10495F000AD8A423D04F0E000172651FD0540E0049
:10496F0001725DD8B01AD0B00E0001722500016837
:10497F006F0001696BFF0E6923000E00016B6F035F
:10498F000E00016A6FE9EC14F0BC0E0001682500FF
:10499F00016E6F7F0E000169214DD0000E00016383
:1049AF006F0C0E0001626F000172C060F0000161B8
:1049BF006B71EC20F0000160C068F0000161C0690C
:1049CF00F0000E00016B6F240E00016A6FE9EC140A
:1049DF00F08A0E0001706F770E716F000168510041
:1049EF000170270001695100017123000E0001635E
:1049FF006F0C0E0001626F000172C060F000016168
:104A0F006B06EC1EF0000160C068F0000161C06928
:104A1F00F0000E00016B6F030E00016A6FE9EC14DA
:104A2F00F0000168510001702500016E6F000169EF
:104A3F00510001712100016F6F1200040120511FFD
:104A4F000B016E0104D8A47BD004012451D8A477A4
:104A5F00D004012151060AD8B41FD027D05304D84F
:104A6F00A424D07D0E0001F66FE20E0001F56F0059
:104A7F000E0001FA6F090E0AD07C0E0001F66FDCF2
:104A8F000E0001F56F000E0001FA6F400E0001F9E4
:104A9F006FC00E0001F86F09D004012351210AD80D
:104AAF00B4DDD7030AD8B4E8D7010A04012039E8E6
:104ABF0032030B016E0104D8A442D02DD0DFEC13CA
:104ACF00F03ED0000E0001F66F570E0001F56F009B
:104ADF000E0001FA6F010E0001F96FC10E13D080A5
:104AEF000E0001F86F23C457F02AD0000E0001F614
:104AFF006F560E0001F56F000E0001FA6F010E00E8
:104B0F0001F96F810E0001F86F1AD0800E0001F8C5
:104B1F006F22C456F014D004012151010AD8B40FEA
:104B2F00D0030AD8B4CED7010AD8B4DFD70A0AD82F
:104B3F00B4C5D7030AD8B4D3D7010AD8B4E6D7126D
:104B4F00000001746F000174512BEC1CF000017513
:104B5F006F000174C060F00001616B000E00016313
:104B6F006F0C0E0001626F71EC20F00001605100BC
:104B7F0001766F000174C060F00001616B000E00E0
:104B8F0001636F0C0E0001626F06EC1EF0000160F6
:104B9F00510001776F00017551D8B443D0000175F2
:104BAF005156D0000176510C0DCF0E0001726F756A
:104BBF000E1FD0000176510C0D6F0E0001726F7534
:104BCF000E17D0000176510C0D2F0E0001726F766B
:104BDF000E0FD0000176510C0D8F0E0001726F7603
:104BEF000E07D0000176510C0DEF0E0001726F769B
:104BFF000E736FF35000017227F4500001732300FE
:104C0F00017751010DF35000017227F45000017329
:104C1F002372C0F6FF73C0F7FF08000001F5CF75D0
:104C2F00F012D00001E251000AD8B4DBD7010AD844
:104C3F00B4B8D7030AD8B4BDD7010AD8B4C2D707BE
:104C4F000AD8B4C7D7CED7000175510AEC1AF012A3
:104C5F00000001E505D8B46DBA07D0000E686E6983
:104C6F00806988020E0001E56F68B469A403D068FB
:104C7F009404EC15F06DB282D068B069A007D036FD
:104C8F00EC29F0A08A040E0001E56F689068B869FE
:104C9F00A803D09FEC13F0689868AC18D069AC0EDD
:104CAF00D0000E166E730E156E000E186E000E17D6
:104CBF006E000E1A6E010E196E61EC18F0689C48AA
:104CCF0050D8A44806486602D042EC1DF068BA6975
:104CDF00AA02D076EC15F068B269A20FD07F0E163B
:104CEF006E1568000E186E000E176E000E1A6E010C
:104CFF000E196E61EC18F0000E6A6E040E0001E5DD
:104D0F005DD8B069A63BD0000E2A6E35D068A636A6
:104D1F00D06CCF55F05530E832E8320F0B4B6E6840
:104D2F009655B409D04B50010D0001DE0EF324D976
:104D3F006E0001000E08D04B50010D0001DC0EF388
:104D4F0024D96E0001000EF420DA6E0001DF704BE3
:104D5F006603D005EC20F00ED0000E166E720E1505
:104D6F006E000E186E550E176E000E1A6E000E198D
:104D7F006E61EC18F02A2A030E2A64C8D7A19A1282
:104D8F00007F0E0001626F6E0E0001616FA6EC16C0
:104D9F00F0FE0EF66E170EF76E09000001F5CF60EC
:104DAF00F00A000001F5CF61F0CFEC14F01AEC1708
:104DBF00F0280E1AEC17F07F0E0001626FD40E0070
:104DCF0001616FA6EC16F0000E0001616F000E007E
:104DDF0001606FCFEC14F01AEC17F0370E1AEC17C6
:104DEF00F0000E0001616F010E0001606FCFEC1437
:104DFF00F01AEC17F0000E0001616F050E00016054
:104E0F006FCFEC14F01AEC17F0280E1AEC17F07E97
:104E1F000E0001626F210E0001616FA6EC16F058B3
:104E2F00EC13F07F0E0001626FDE0E0001616FA6C2
:104E3F00EC16F0F2EC12F07F0E0001626FE20E0042
:104E4F0001616FA6EC16F025EC13F07F0E000162E6
:104E5F006FE60E0001616FA6EC16F003EC13F07F06
:104E6F000E0001626FEA0E0001616FA6EC16F047AB
:104E7F00EC13F07F0E0001626FEE0E0001616FA662
:104E8F00EC16F014EC13F07F0E0001626FF20E00BF
:104E9F0001616FA6EC16F036EC13F07F0E00016285
:104EAF006FDA0E0001616FA6EC16F069EC13F012C9
:104EBF000020EE01F03D50D9263E50DA22DF50029D
:104ECF006E02500001D45D000E0001D559D8A0D458
:104EDF00C002F002500001D45F000E0001D55B004C
:104EEF000E016E14D00150010D0401280EF324D9C8
:104EFF006E0401040EF420DA6ED0C0E1FFD1C0E2DF
:104F0F00FFDFCFE7FF0001D04BD12B012A02500169
:104F1F005CD8A0E8D70001D551D411D8B42BD0203C
:104F2F00EE01F03F50D9264050DA22080EDF6E20F6
:104F3F00EE02F03F50D9264050DA22280EDE6E04E2
:104F4F000EDD6E3DC0D9FF3EC0DAFFDFBC06D03F9D
:104F5F00C0D9FF40C0DAFF480E05D03FC0D9FF408F
:104F6F00C0DAFF080EDF6E3FC0D9FF40C0DAFF0086
:104F7F000EDB8E38D020EE01F03F50D9264050DAAC
:104F8F0022080EDF6E20EE02F03F50D9264050DA95
:104F9F0022200EDE6E040EDD6E3FC0D9FF40C0DA58
:104FAF00FF040EDF6E3FC0D9FF40C0DAFF000EDBFB
:104FBF008E0001D751D611D8B40FD0000120EED6F4
:104FCF00F001D80AD00500FA6EDE50FD6EDE50FEFD
:104FDF006EF850FF6EFA5012000001D39F45660223
:104FEF00D042EC1DF0120000017C6FFE0EF66E1722
:104FFF000EF76E0900F5CF79F00900F5CF7AF002C0
:10500F000E0001795D000E7A59D8A020D000017CE6
:10501F00510C0D0F0E0001796F750E7A6FF3500062
:10502F00017927F45000017A2300017851010DF323
:10503F005000017927F45000017A2379C0F6FF7AE6
:10504F00C0F7FF08000001F5CF7BF008D000017C0E
:10505F00510C0DF3500001782500017B6F00017892
:10506F0051010D0101C40EF324D96E0101010EF49B
:10507F0020DA6EDF2A00017C51010D0101D80EF3F9
:10508F0024D96E0101010EF420DA6EDF2A00017BB4
:10509F0051A8EC25F000017D6FDF0E00017D651B2F
:1050AF00D0E80E00017D5DD8B016D07DC079F0201C
:1050BF000E00017927010E00017A6F0001792B0391
:1050CF00D00001D8907A370001792FFAD700017AF2
:1050DF00510001ED1323D000017D51F00AD8A40334
:1050EF00D00101D1811BD00001FC51800A00017950
:1050FF006F080E800A0001795DD8B010D00001FC56
:10510F0051010D0101D00EF324D96E0101010EF4EE
:10511F0020DA6E00017BC0DFFF0001FC2B120004C0
:10512F00012051800AD8A499D0C00E0001F86F89D0
:10513F00D07F0E0001F66FAA0E0001F56F000E0072
:10514F0001FA6F120E0001F96F88D0040122677502
:10515F00D004012251020D880EF324F66E770EF45F
:10516F0020F76E09000001F5CFF5F00A000001F5F8
:10517F00CFF6F0020E0001F525016E000E0001F6CC
:10518F0021026E01C0F6FF02C0F7FFF86A070EF7A3
:10519F006403D00800F55005D0F6CFE1FFF7CFE25A
:1051AF00FFE7500001F96F030E0001F525016E00B6
:1051BF000E0001F621026E01C0F6FF02C0F7FFF8E4
:1051CF006A070EF76403D00800F55005D0F6CFE15B
:1051DF00FFF7CFE2FFE7500001FA6F3FD0030E0455
:1051EF0001225DD8B02AD004012251020D7E0EF3A8
:1051FF0024F66E770EF420F76E09000001F5CFF557
:10520F00F00A000001F5CFF6F00001F5C0F6FF003F
:10521F0001F6C0F7FFF86A070EF76403D00800F530
:10522F005005D0F6CFE1FFF7CFE2FFE750016E0157
:10523F00500001F96F0001FA6B10D0000E0001F859
:10524F006F0CD004012351010AD8B472D7030AD8C6
:10525F00B47CD7010AD8B4C2D7F0D71200A09A00F5
:10526F000E6A6E000E686E000E706E0F0E026E717B
:10527F000E016E000E046E000E036E000E066E0120
:10528F000E056EC9EC13F0160E6F6E9F0E6B6E7BD4
:10529F000E696E000E096E0FD00950040D04010047
:1052AF000EF324D96E0401040EF420DA6EDE6ADEEA
:1052BF006ADE6ADD6A092A070E0964EED76D8C0073
:1052CF000E6E6E6D986D9C0DD06896000E0001F8F5
:1052DF006F000E0001D36F000E0001D56F000E009E
:1052EF0001D46F68B6F1D7010E466E010E476E00FE
:1052FF000E436E000E446E000E0001E46F000E09A7
:10530F006E33D00950020D0001D80EF324D96E0070
:10531F0001000EF420DA6E000EDE6E000EDD6E0957
:10532F0050020D390EF324D96E000EF420DA6E0000
:10533F000EDE6E000EDD6E0950010D0001DC0EF366
:10534F0024D96E0001000EF420DA6E000EDF6E0914
:10535F0050010D0001DE0EF324D96E0001000EF492
:10536F0020DA6E000EDF6E092A010E0964CAD70417
:10537F0001040E0001D96F0401080E0001D86F1649
:10538F000E706E040E0401036F200E0401026F08ED
:10539F000E0401016F040E0401006F0401008F0061
:1053AF000E536E000E0001E56F1200A09A000E6AF8
:1053BF006E000E686E000E706E0F0E0001616F7141
:1053CF000E0001606F000E0001636F000E0001629E
:1053DF006F000E0001656F010E0001646F20EC1568
:1053EF00F0160E6F6E9F0E6B6E7B0E696E000E00C9
:1053FF0001686F11D000016851040D0401000EF314
:10540F0024D96E0401040EF420DA6EDE6ADE6ADE41
:10541F006ADD6A0001682B070E00016865EBD76D26
:10542F008C000E6E6E6D986D9C0DD06896000E0000
:10543F0001F86F000E0001D36F000E0001D56F0051
:10544F000E0001D46F68B6F1D7010E466E010E47FC
:10545F006E000E436E000E446E000E0001E46F00EE
:10546F000E0001686F38D000016851020D0001D89D
:10547F000EF324D96E0001000EF420DA6E000EDE5A
:10548F006E000EDD6E00016851020D390EF324D946
:10549F006E000EF420DA6E000EDE6E000EDD6E0072
:1054AF00016851010D0001DC0EF324D96E000100DB
:1054BF000EF420DA6E000EDF6E00016851010D0050
:1054CF0001DE0EF324D96E0001000EF420DA6E0017
:1054DF000EDF6E0001682B010E00016865C4D70452
:1054EF0001040E0001D96F0401080E0001D86F16D8
:1054FF000E706E040E0401036F200E0401026F087C
:10550F000E0401016F040E0401006F0401008F00EF
:10551F000E536E000E0001E56F1200D8D00001A6E9
:10552F00C084F00001A5C083F00001A8C086F00080
:10553F0001A7C085F00001AAC088F00001A9C087AB
:10554F00F07A0E00018A6FF60E0001896F7B0E0054
:10555F00018C6F4A0E00018B6F7B0E00018E6F9EC8
:10556F000E00018D6F37EC37F0C3D00001A6C08459
:10557F00F00001A5C083F00001A8C086F00001A7CC
:10558F00C085F00001AAC088F00001A9C087F0799A
:10559F000E00018A6F520E0001896F790E00018C87
:1055AF006FA60E00018B6F790E00018E6FFA0E0041
:1055BF00018D6F37EC37F09CD00001A6C084F0004E
:1055CF0001A5C083F00001A8C086F00001A7C08527
:1055DF00F00001AAC088F00001A9C087F0780E0082
:1055EF00018A6FAA0E0001896F780E00018C6FFE81
:1055FF000E00018B6F780E00018E6FFE0E00018D75
:10560F006F37EC37F075D00001A6C084F00001A50C
:10561F00C083F00001A8C086F00001A7C085F0008C
:10562F0001AAC088F00001A9C087F07A0E00018A94
:10563F006F4E0E0001896F7A0E00018C6FA20E0063
:10564F00018B6F7A0E00018E6FA20E00018D6F37E6
:10565F00EC37F04ED00001A6C084F00001A5C08346
:10566F00F00001A8C086F00001A7C085F00001AAD4
:10567F00C088F00001A9C087F07B0E00018A6FF28D
:10568F000E0001896F7C0E00018C6F460E00018B9E
:10569F006F7C0E00018E6F460E00018D6F37EC3759
:1056AF00F027D00001A6C079F00001A5C078F00066
:1056BF0001A8C07BF00001A7C07AF00001AAC07D4D
:1056CF00F00001A9C07CF029EC24F012D00001EC0D
:1056DF0051010AD8B44AD7030AD8B46ED7010AD8F1
:1056EF00B41DD7070AD8B48FD7010AD8B4B3D7D906
:1056FF00D71200000E01019F6F000E01019E6F0077
:10570F000E0501086F1E0E096E010E39EC16F00022
:10571F000E016E0501050E036E0501080E026E01E6
:10572F000E046E010EE1EC1CF001C0A0F102C0A14D
:10573F00F1FE0EF66E170EF76E0900F5CF0FF0099A
:10574F0000F5CF10F00F50030A1010D8A440D00F5F
:10575F000E01013B6F960E01013A6F000E116E178D
:10576F00D01150010D0101840EF324D96E010101F6
:10577F000EF420DA6E1150010D01017C0EF324E1BD
:10578F006E0101010EF420E26EDFCFE7FF112A0751
:10579F000E1164E6D7000E126E17D01250010D01D4
:1057AF00015C0EF324D96E0101010EF420DA6E12A2
:1057BF0050010D0101500EF324E16E0101010EF4B1
:1057CF0020E26EDFCFE7FF122A0B0E1264E6D7FE40
:1057DF000EF66E170EF76E0900F5CF0FF00900F5F4
:1057EF00CF10F0040E0F5C000E1058D8A080D00020
:1057FF000E136E2FD01350020D0101400EF324D95A
:10580F006E0101010EF420DA6E1350020D0101300A
:10581F000EF324E16E0101010EF420E26EDECFE6FD
:10582F00FFDDCFE5FF1350010D01018C0EF324D9DD
:10583F006E0101010EF420DA6E1350010D01017C8F
:10584F000EF324E16E0101010EF420E26EDFCFE7CB
:10585F00FF132A070E1364CED7000E146E2FD01429
:10586F0050020D0101180EF324D96E0101010EF43F
:10587F0020DA6E1450020D0101000EF324E16E01C7
:10588F0001010EF420E26EDECFE6FFDDCFE5FF145F
:10589F0050010D0101680EF324D96E0101010EF4C0
:1058AF0020DA6E1450010D0101500EF324E16E0148
:1058BF0001010EF420E26EDFCFE7FF142A0B0E1466
:1058CF0064CED7FE0EF66E170EF76E0900F5CF0FEA
:1058DF00F00900F5CF10F0050E0F5C000E1058D830
:1058EF00A006D0010E01015A6F020E01015B6F1766
:1058FF000ED2EC12F0A4EC12F001C0A4F102C0A57C
:10590F00F1120004012205D8A412D0040120511F66
:10591F000B0009D8A40CD00001F88F04012151030A
:10592F000AD8A402D0010E01D0000E0001E36F04CB
:10593F0001226740D1040120511F0B020AD8A43A5B
:10594F00D1040124510F0B0009D8B434D104012420
:10595F00510F0B1D6E020E1D5CD8B02CD10001E54E
:10596F0051200AD8A427D10001F88F040124BF1DAC
:10597F00D0040124510F0B1D6E1D50020D390EF373
:10598F0024D96E000EF420DA6EDECF23F0DDCF24A3
:10599F00F0040124510F0B1D6E1D50010D0001DE8F
:1059AF000EF324D96E0001000E1ED0040124510FF6
:1059BF000B1D6E1D50020D0001D80EF324D96E0081
:1059CF0001000EF420DA6EDECF23F0DDCF24F004D9
:1059DF000124510F0B1D6E1D50010D0001DC0EF344
:1059EF0024D96E0001000EF420DA6EDF50226E22F1
:1059FF00B002D0239401D02384040124BF0BD00420
:105A0F000124510F0B1D6E1D50020D390EF324D9B9
:105A1F006E000E0CD0040124510F0B1D6E1D500291
:105A2F000D0001D80EF324D96E0001000EF420DA18
:105A3F006E23C0DEFF24C0DDFF04012151030AD80D
:105A4F00A433D023C0D9FF24C0DAFFDFAE20D004A7
:105A5F000124BF0DD0040124510F0B1D6E1D5001E9
:105A6F000D0001DE0EF324D96E0001000E0CD004E0
:105A7F000124510F0B1D6E1D50010D0001DC0EF3A3
:105A8F0024D96E0001000EF420DA6E0001DF8223AC
:105A9F00C0D9FF24C0DAFF000EDB8423C0D9FF2456
:105AAF00C0DAFF000EDB8E86D0040E231A23C0D976
:105ABF00FF24C0DAFFDFAE1BD023C0D9FF24C0DA2A
:105ACF00FF7F0EDF1623C0D9FF24C0DAFF000EDBE5
:105ADF008C000E166E050E156E24C018F023C0171D
:105AEF00F0000E1A6E020E196E61EC18F006D0233C
:105AFF00C0D9FF24C0DAFF000EDB8C040E231A225C
:105B0F00B206D023C0D9FF24C0DAFFDFAE35D004F0
:105B1F000124BF0DD0040124510F0B1D6E1D500128
:105B2F000D0001DE0EF324D96E0001000E0CD0041F
:105B3F000124510F0B1D6E1D50010D0001DC0EF3E2
:105B4F0024D96E0001000EF420DA6E0001DF9223DB
:105B5F00C0D9FF24C0DAFF3B0EDF16000E166E050C
:105B6F000E156E24C018F023C017F0000E1A6E0227
:105B7F000E196E61EC18F006D023C0D9FF24C0DADD
:105B8F00FF3B0EDF16040124510F0B1D6E1D50013C
:105B9F000D700E1E6E0F0E1F6EF3501E26F4501F4B
:105BAF00221EC020F01FC021F020C0D9FF21C0DA73
:105BBF00FFFE0EDF1612000001ACC061F00001AB5A
:105BCF00C060F00001AEC063F00001ADC062F00034
:105BDF000E0001656F080E0001646F79EC19F0007B
:105BEF0001615100016011D8A402D0000E9FD100B5
:105BFF0001B0C061F00001AFC060F0000E000163A2
:105C0F006F000E0001626F000E0001656F080E003D
:105C1F0001646F20EC15F0000120EE01F00001ABE4
:105C2F0051D9260001AC51DA22DF500001B16F00CB
:105C3F0001B1A122D1ABC0D9FFACC0DAFFDF500058
:105C4F0001B56F020E0001B76F010E0001BB6F02AD
:105C5F000E0001B86FFFD00001B851010DF35000D5
:105C6F0001AB25D96EF4500001AC21DA6EDF500084
:105C7F0001B66F0001B651A6EC24F000016EC0B35F
:105C8F00F000016FC0B4F0000E0001B96FD8D00062
:105C9F0001B951010D0001B3C0B1F00001B4C0B2A0
:105CAF00F0F3500001B127F4500001B223B1C0F658
:105CBF00FFB2C0F7FF08000001F5CFBAF0020E00E7
:105CCF0001AD250001606F000E0001AE21000161E2
:105CDF006F0001B6C062F00001636B000E0001653A
:105CEF006F060E0001646FCDEC18F00001615100DA
:105CFF00016011D8A402D0010E01D0000E0001BC2A
:105D0F006F6FD00001BC51D8B498D0C8EC26F037D3
:105D1F00D00001BC51D8B491D086EC14F030D00033
:105D2F0001BC51D8B48AD0F6EC13F029D00001BCD5
:105D3F0051D8B483D03EEC14F022D00001BC51D81E
:105D4F00B47CD00EEC14F01BD00001BC51D8B4754C
:105D5F00D06EEC14F014D00001BC51D8B46ED02624
:105D6F00EC14F00DD00001BC51D8B467D056EC1430
:105D7F00F006D00001BC51D8B460D09EEC14F004F2
:105D8F000E0001BB6F5AD00001B58157D0110E0024
:105D9F0001B51353D00001B58350D00001B58B4D21
:105DAF00D0ABC0D9FFACC0DAFFDF500001686FBCC9
:105DBF00C069F00001BA513EEC19F00001BA6F0052
:105DCF0001B751010DF3500001AF25D96EF450000A
:105DDF0001B021DA6E0001BAC0DFFF0001B72B2D31
:105DEF00D00001BA51000AD8B428D03A0AD8B489E1
:105DFF00D7010AD8B48DD7070AD8B491D7010AD8DA
:105E0F00B495D7030AD8B499D7010AD8B49DD77FD0
:105E1F000AD8B4A1D7010AD8B4A5D7030AD8B4A910
:105E2F00D7A20AD8B4B0D7010AD8B4B4D7050AD8C4
:105E3F00B4ADD7010AD8B4B1D7B3D70001B92B038A
:105E4F000E0001B95DD8B004D0070E0001B7651F71
:105E5F00D70001B82B080E0001B85DD8B005D000EF
:105E6F0001BB51040AD8A4F7D6AFC0D9FFB0C0DA2E
:105E7F00FF0001B5C0DFFF36D00001ACC061F000FC
:105E8F0001ABC060F005EC19F00009D8B415D000D3
:105E9F0001ACC0A6F00001ABC0A5F00001AEC0A8D8
:105EAF00F00001ADC0A7F00001B0C0AAF00001AF33
:105EBF00C0A9F095EC2AF014D00001ACC079F00025
:105ECF0001ABC078F00001AEC07BF00001ADC07A2D
:105EDF00F00001B0C07DF00001AFC07CF029EC24D0
:105EEF00F00001BB6F0001BB05D8B40AD00001BBA5
:105EFF0051030AD8B405D00001BB51040AD8A41429
:105F0F00D00001AEC061F00001ADC060F00001AC87
:105F1F00C063F00001ABC062F0000E0001656F08B6
:105F2F000E0001646FB0EC23F00001BB51120002B0
:105F3F000E0001726FC7D100017251010DF35000B5
:105F4F00016C25D96EF45000016D21DA6E680E0CCC
:105F5F00D000017251010DF35000016C25D96EF480
:105F6F005000016D21DA6E690EDF6EAAD100017249
:105F7F0051010DF35000016C25D96EF45000016DE5
:105F8F0021DA6EDF508A0AD8B4B9D0010AD8B4B674
:105F9F00D01B0AD8B4D0D7010AD8B4DAD791D10020
:105FAF0001EB51020AD8B405D00001EB51050AD814
:105FBF00A487D16CC0D9FF6DC0DAFF000EDB84005F
:105FCF00017251010DF35000016C250001606FF457
:105FDF005000016D210001616F00017251010D0030
:105FEF00016CC06EF000016DC06FF0F35000016ED8
:105FFF0027F45000016F23010E00016E27000E6F72
:10600F00236EC062F06FC063F00001725100017027
:10601F006F716B0001701F711F704B712B070E009A
:10602F000170250001646F000E00017121000165F0
:10603F006FB0EC23F0000120EE07F000016C51D996
:10604F002600016D51DA22000EDF6E000172073853
:10605F00D100017251010DF35000016C25D96EF47E
:10606F005000016D21DA6EDF50650AD8B498D7EF72
:10607F000AD8B444D0010AD8B441D022D100017259
:10608F0051010DF35000016C25D96EF45000016DD4
:10609F0021DA6E2C0E72D000017251010DF35000F7
:1060AF00016C25D96EF45000016D21DA6E2A0E6550
:1060BF00D000017251010DF35000016C25D96EF41F
:1060CF005000016D21DA6EDF508A0AD8B417D00163
:1060DF000AD8B414D01B0AD8B4D1D7010AD8B4DB6C
:1060EF00D7EFD000017251010DF35000016C25D98B
:1060FF006EF45000016D21DA6E350E86D0000172FC
:10610F0051010DF35000016C25D96EF45000016D53
:10611F0021DA6E2C0E29D700017251010DF35000B8
:10612F00016C25D96EF45000016D21DA6EDF508AB3
:10613F000AD8B4E4D7010AD8B4E1D71B0AD8B4D12E
:10614F00D7010AD8B4CED7BCD000017251010DF3DC
:10615F005000016C25D96EF45000016D21DA6E8A62
:10616F000E0CD000017251010DF35000016C25D9B6
:10617F006EF45000016D21DA6E8B0EDF6E6CC0D99C
:10618F00FF6DC0DAFF030EDF129BD00001725101C9
:10619F000DF35000016C25D96EF45000016D21DA1A
:1061AF006EDF50900AD8B4D0D7010AD8B4DAD788A6
:1061BF00D000017251010DF35000016C25D96EF41E
:1061CF005000016D21DA6E350ECFD60001725101EC
:1061DF000DF35000016C25D96EF45000016D21DADA
:1061EF006EDF50900AD8B4E4D7010AD8B4E1D7686B
:1061FF00D000017251010DF35000016C25D96EF4DE
:10620F005000016D21DA6E2C0EDF6E6CC0D9FF6D60
:10621F00C0DAFF000EDB8454D000017251010DF380
:10622F005000016C25D96EF45000016D21DA6EDF3C
:10623F0050900AD8B4DDD7010AD8B4DAD741D000CC
:10624F00017251010DF35000016C25D96EF450000D
:10625F00016D21DA6E2C0EDF6E6CC0D9FF6DC0DAC6
:10626F00FF000EDB822DD000017251010DF35000A3
:10627F00016C25D96EF45000016D21DA6EDF50905C
:10628F000AD8B4DDD7010AD8B4DAD71AD00001F191
:10629F0051000AD8B46BD6010AD8B4DAD6030AD89B
:1062AF00B407D7010AD8B437D7070AD8B46ED701C5
:1062BF000AD8B48BD7030AD8B4AFD7010AD8B4D34E
:1062CF00D70001722B070E00017265E0D712000094
:1062DF000E0001C16F37EC23F00009D8B410D09431
:1062EF00D10001FC51010D0101D00EF324D96E0133
:1062FF0001010EF420DA6E0E0EDF6E0001FC2B0092
:10630F0001FC51800A780FD8A0EBD70001E75106A6
:10631F000D0101A60EF3240001606F0101010EF4BF
:10632F00200001616F0101010E0001636F0101D2B5
:10633F000E0001626F000E0001656F060E00016412
:10634F006FB0EC23F0EDC0D0F10001F351D8B423BE
:10635F00D00101010E0001616F0101D00E0001603B
:10636F006F05EC19F00009D8B416D00001F25101F5
:10637F0001D0130001EEB306D00001EDA303D0024C
:10638F000E0001F21B0001EEBB06D00001EDAB03C6
:10639F00D0200E0001F21BEDC0EEF00001E651001F
:1063AF00080001E725050F0001C36F040E0001C3AC
:1063BF006503D0050E0001C35F0001C351040F0038
:1063CF0001C56F040E0001C56503D0050E0001C5A0
:1063DF005F020E0001FC6F000E0001C46F53D0006E
:1063EF0001C351060DA60E0001BF6F010EC06FF362
:1063FF00500001BF27F4500001C0230001C4510118
:10640F000DF3500001BF25D96EF4500001C021DA01
:10641F006EDF500001C26F0001C551060DA60E00C0
:10642F0001BF6F010EC06FF3500001BF27F4500082
:10643F0001C023BFC060F0C0C061F00001C2C062E4
:10644F00F00001636B000E0001656F060E00016422
:10645F006FCDEC18F00001615100016011D8B4103C
:10646F00D00001FC51010D0101D00EF324D96E01B2
:10647F0001010EF420DA6E0001C2C0DFFF0001FC43
:10648F002B0001C42B050E0001C465A9D70FD00046
:10649F0001FC51010D0101D00EF324D96E01010150
:1064AF000EF420DA6E0E0EDF6E0001FC2B0001FCE5
:1064BF0051800A780FD8A0EBD70001EAA502D001CE
:1064CF0001D1810101010E0001616F0101D00E00A8
:1064DF0001606F0101010E0001636F0101960E0053
:1064EF0001626F000E0001656F080E0001646F7985
:1064FF00EC19F00001615100016011D8B47CD0019A
:10650F0001010E0001616F0101D20E0001606F01E8
:10651F0001010E0001636F0101980E0001626F000F
:10652F000E0001656F060E0001646F79EC19F00023
:10653F0001615100016011D8A40FD00101D2510E99
:10654F000AD8B40AD00101D16707D0D0C1BFF02259
:10655F000E0001BF17D8B421D00101D2510E0AD8B5
:10656F00B403D0000E0001F26F0101010E0001AC67
:10657F006F0101D00E0001AB6F0101010E0001AEE2
:10658F006F0101960E0001AD6F0001BEC0B0F000AB
:10659F0001BDC0AFF0E3EC2DF02CD001019751D825
:1065AF00B404D00101D151D8B426D0010196A30370
:1065BF00D00101D0A320D0010196AB03D00101D0AF
:1065CF00AB1AD00101010E0001AC6F0101D00E001A
:1065DF0001AB6F0101010E0001AE6F0101960E00BC
:1065EF0001AD6F0001BEC0B0F00001BDC0AFF0E360
:1065FF00EC2DF00001C16F0001BEC06DF00001BDB8
:10660F00C06CF09FEC2FF033D00001E751040F0066
:10661F0001C56F040E0001C56503D0050E0001C54D
:10662F005F0001E751060D0101A60EF32400016082
:10663F006F0101010EF4200001616F0001C55106C9
:10664F000DA60E0001BF6F010EC06FF3500001BF0A
:10665F0027F4500001C023BFC062F0C0C063F00038
:10666F000E0001656F060E0001646FB0EC23F000A1
:10667F0001E72B040E0001E76503D0000E0001E7D0
:10668F006F020E0001FC6F000E0001ED6F000E0196
:10669F0001D16F0001C15112000001FB51020AD854
:1066AF00B438D00001FB51030AD8B433D00101A490
:1066BF00C1C6F00101A5C1C7F00001C61FC71FC6A3
:1066CF004BC72BB6EC12F00001C65100016027003A
:1066DF0001C7510001612300016151800A800F8DB4
:1066EF000ED8B40001605DD8A0E1D7B6EC12F0006F
:1066FF000160C0A4F1000161C0A5F10001E02B0011
:10670F0001E0C0C6F00001C76BC6BFC7070001C6D6
:10671F00B1A7D101019F519E11D8B413D09EC1D9F9
:10672F00FF9FC1DAFFDFAE04D00001C66BC62B029C
:10673F00D00001C66B0001C6510001C96F0001CA2C
:10674F006B06D0000E0001CA6F000E0001C96F006A
:10675F0001CA51C911D8A44AD10001FB51030AD86B
:10676F00A419D005010251D8B40AD0B4EC13F00526
:10677F00010219D8A404D0000E0501026F1CD15DCF
:10678F00EC16F00501026F0501026715D1000E002E
:10679F0001FB6F11D1070E0001CF6F82D00001CF27
:1067AF0051010D01017C0EF324D96E0101010EF48C
:1067BF0020DA6EDF50FF0A0001C66F0001CF5102D1
:1067CF000D0101300EF324D96E0101010EF420DA10
:1067DF006EDECFC7F0DDCFC8F0C7C0D9FFC8C0DAB3
:1067EF00FF0001C651DF16000E0001CE6F2FD00043
:1067FF0001CE51010D0101500EF324D96E0101019B
:10680F000EF420DA6EDF500001C66F0001CE510288
:10681F000D0101000EF324D96E0101010EF420DAEF
:10682F006EDECFC7F0DDCFC8F0C7C0D9FFC8C0DA62
:10683F00FFDF500001C6150009D8A406D0CEC078DE
:10684F00F00001CF51FBEC27F00001CE2B0B0E0017
:10685F0001CE65CDD70001CF51010D01017C0EF3A3
:10686F0024D96E0101010EF420DA6EDF500001C64B
:10687F006F0001CF51020D0101300EF324D96E01CB
:10688F0001010EF420DA6EDECFC7F0DDCFC8F0C7FE
:10689F00C0D9FFC8C0DAFF0001C651DF120001CF17
:1068AF00070001CFAF7BD70501050E0001BE6F05B5
:1068BF0001000E0001BD6F6FEC31F00001FB6F6D39
:1068CF00D00501050E0001616F0501100E0001607A
:1068DF006F000E0001636F000E0001626F000E006B
:1068EF0001656F060E0001646F20EC15F064D00097
:1068FF000E0001CD6F10D00001CD51010D05010229
:10690F000EF324D96E0501050EF420DA6EDF501A4E
:10691F00EC17F00001CD2B050E0001CD65ECD7066D
:10692F000EC8EC12F00501026F0501050E000161A2
:10693F006F0501030E0001606F000E0001636F0011
:10694F000E0001626F000E0001656F050E000164FD
:10695F006F20EC15F030D0030E0001FB6F000E0519
:10696F0001006F800EC8EC12F00501026F050105E2
:10697F000E0001616F0501030E0001606F000E0034
:10698F0001636F000E0001626F000E0001656F055D
:10699F000E0001646F20EC15F00ED00001FB5101C9
:1069AF000AD8B409D0030AD8B48BD7010AD8B49F38
:1069BF00D7070AD8B4D0D70001FB51D8B417D001EC
:1069CF000E0001606F0501050E0001626F050100E9
:1069DF000E0001616F080E0001636F010E46EC227D
:1069EF00F0000160C09EF1000161C09FF10101A1A3
:1069FF0051A011D8B413D0A0C1D9FFA1C1DAFFDFC4
:106A0F00AE04D00001C66BC62B02D00001C66B00CE
:106A1F0001C6510001CB6F0001CC6B06D0000E00F8
:106A2F0001CC6F000E0001CB6F0001CC51CB11D800
:106A3F00A417D0000E0001606F0501050E00016262
:106A4F006F0501080E0001616F010E0001636F01F8
:106A5F000E46EC22F0000160C0A0F1000161C0A160
:106A6F00F112000001826FA10E0001825DD8B09873
:106A7F00D0000182C060F00001616B000E00016365
:106A8F006F070E0001626F71EC20F0D8900001606B
:106A9F0037000161374E0E0001602500017F6F7DC9
:106AAF000E000161210001806F000E0001816F2334
:106ABF00D000018151010D00017FC07AF0000180EB
:106ACF00C07BF0F35000017A27F45000017B237A4A
:106ADF00C0F6FF7BC0F7FF00018151010DF350009D
:106AEF00017825D96EF45000017921DA6E0800F58E
:106AFF00CFDFFF0001812B020E0001815DD8B0189E
:106B0F00D000018151010D00017FC07AF00001809A
:106B1F00C07BF0F35000017A27F45000017B237AF9
:106B2F00C0F6FF7BC0F7FF0800F5500009D8A4C0DE
:106B3F00D7000182C060F00001616B000E0001639D
:106B4F006F070E0001626F06EC1EF0770E000160FA
:106B5F0025F66E770E00016121F76E00018151015C
:106B6F000DF35000017825D96EF45000017921DA28
:106B7F006E0800F5CFDFFF0DD000018151010DF33D
:106B8F005000017825D96EF45000017921DA6E009A
:106B9F000EDF6E0001812B020E00018165EDD75EC5
:106BAF00D1A00E000182652FD0B70E0001825DD8F3
:106BBF00B02AD0000179C06FF0000178C06EF05F8D
:106BCF000E000182250001686F0001696BFF0E69DD
:106BDF0023000E00016B6F030E00016A6FE9EC14C6
:106BEF00F09A0E000168250001706F7C0E0001699C
:106BFF00210001716F000E0001736F030E0001720F
:106C0F006F2CEC18F02BD1C70E000182653FD0E13D
:106C1F000E0001825DD8B03AD0000179C06FF0004C
:106C2F000178C06EF0700E00017A6FFE0E7B6F0060
:106C3F0001825100017C6F7D6BD89000017C377D04
:106C4F003700017A5100017C2700017B5100017D43
:106C5F00231C0E00017C250001706F7D0E00017D4D
:106C6F00210001716F000E0001736F020E0001729F
:106C7F006F2CEC18F0000120EE02F000017851D9D2
:106C8F002600017951DA22000EDF6EE8D0E50E0002
:106C9F00018265D0D0F20E0001825DD8A065D0CA06
:106CAF00D01A0E000182250001686F0001696BFF89
:106CBF000E6923000E00016B6F030E00016A6FE96E
:106CCF00EC14F08F0E0001682500017F6F7E0E47D8
:106CDF00D01A0E000182250001686F0001696BFF59
:106CEF000E6923000E00016B6F030E00016A6FE93E
:106CFF00EC14F0470E0001682500017F6F7E0E2F08
:106D0F00D01A0E000182250001686F0001696BFF28
:106D1F000E6923000E00016B6F030E00016A6FE90D
:106D2F00EC14F06B0E0001682500017F6F7E0E17CB
:106D3F00D01A0E000182250001686F0001696BFFF8
:106D4F000E6923000E00016B6F030E00016A6FE9DD
:106D5F00EC14F0FB0E0001682500017F6F7E0E0022
:106D6F000169210001806F0FD00001E851000AD89E
:106D7F00B4DFD7010AD8B4C4D7030AD8B491D70166
:106D8F000AD8B4A6D7D5D7000E0001816F020E0026
:106D9F0001816501D063D000018151010D00017F98
:106DAF00C07AF0000180C07BF0F35000017A27F425
:106DBF005000017B237AC0F6FF7BC0F7FF0800006D
:106DCF0001F5CF7EF08CEC13F00009D8A40DD01D87
:106DDF00D0300E07D0320E05D02E0E03D0250E0167
:106DEF00D0260E00017E6F11D000017E51260AD8E9
:106DFF00B4F5D7010AD8B4F4D7080AD8B4E9D71F25
:106E0F000AD8B4E8D7050AD8B4E7D70001815101F1
:106E1F000DF35000017825D96EF45000017921DA75
:106E2F006E00017EC0DFFF0001812B020E00018189
:106E3F0065B2D714D0000179C061F0000178C0604D
:106E4F00F0000E0001636F000E0001626F000E0074
:106E5F0001656F030E0001646F20EC15F0120083C3
:106E6F00C0D9FF84C0DAFFDF5000019F6F020E0010
:106E7F0001A46F010E0001916F83C0D9FF84C0DAA6
:106E8F00FFDF50DD0B0001966F87C0D9FF88C0DA96
:106E9F00FF000196C0DFFF020E0001956FE2D200E6
:106EAF00019551010DF35000018325D96EF4500067
:106EBF00018421DA6EDF500001A16F0001A1C060D3
:106ECF00F00001616B000E0001636F0C0E00016298
:106EDF006F71EC20F0000160510001A06F0001A163
:106EEF00C060F00001616B000E0001636F0C0E00BB
:106EFF0001626F06EC1EF0000160510001976F00F8
:106F0F0001A1512BEC1CF00001A36F0001A351D87C
:106F1F00B425D00001A451010DF35000018725D9EC
:106F2F006EF45000018821DA6E0001A3C0DFFF006C
:106F3F0001A42B000E0001616F500E0001606F0065
:106F4F000E0001636F000E0001626F000E000165FD
:106F5F006F030E0001646F20EC15F009D1000E00D5
:106F6F0001926F9FC08FF0220E00018F1700018FCB
:106F7F0051220AD8A411D04DA203D000019F930C27
:106F8F00D085C0D9FF86C0DAFFDF5000018F6F00B8
:106F9F00018FAB02D000019F9B060E0001A065047C
:106FAF00D0000E0001A26F3AD000019FA30AD000BB
:106FBF0001A0510C0D00018BC08FF000018CC0900F
:106FCF00F016D000019FAB0AD00001A0510C0D00AC
:106FDF00018DC08FF000018EC090F009D00001A08C
:106FEF00510C0D000189C08FF000018AC090F0F3A1
:106FFF005000018F27F45000019023000197510199
:10700F000DF35000018F27F450000190238FC0F62D
:10701F00FF90C0F7FF08000001F5CFA2F00001A21A
:10702F0051D8B431D0D00E0001A26504D0E00E00CB
:10703F0001A26529D0010E0001926F020E00019886
:10704F006F1ED000019851010DF35000018525D915
:10705F006EF45000018621DA6E0001A151DF620D3E
:10706F00D00E0E0001A16F010E0001A06F020E00E5
:10707F0001976F000E0001A26F06D00001982B0739
:10708F000E00019865DED70001A251D8B40CD000D4
:10709F0001000E0001796F00019C0E0001786F0056
:1070AF0001A25139EC35F00001A251D8B403D00040
:1070BF00019C676BD00001A151A8EC25F00001A342
:1070CF006F0001A351D8B4CBD183C0D9FF84C0DAEC
:1070DF00FFDF500001686F020E000185250001607F
:1070EF006F000E000186210001616F0001A3C062D5
:1070FF00F00001636B000E0001656F060E00016466
:10710F006FCDEC18F00001615100016011D8A4029D
:10711F00D0010E01D0000E0001696F0001A3513E96
:10712F00EC19F00001A36F0001A451010DF3500001
:10713F00018725D96EF45000018821DA6E0001A372
:10714F00C0DFFF0001A42B000E0001616F500E0085
:10715F0001606F000E0001636F000E0001626F008F
:10716F000E0001656F030E0001646F20EC15F083B4
:10717F00C0D9FF84C0DAFFDF504D6E83C0D9FF84C2
:10718F00C0DAFFDF500001966F6AD100019251D82B
:10719F00B463D0000E0001996F4CD0000E00019A1D
:1071AF006F33D000019951010D0101E00EF324D985
:1071BF006E0101010EF420DA6E00019A51010D00EB
:1071CF00019C0EF324E16E0001000EF420E26EE745
:1071DF0050DF6218D00101010E0001616F0101E063
:1071EF000E0001606F000E0001636F000E00016260
:1071FF006F000E0001656F030E0001646F20EC1528
:10720F00F0020E7CD100019A2B030E00019A5DD87B
:10721F00B00ED000019A51010D00019C0EF324D93C
:10722F006E0001000EF420DA6EDF50D8A4BAD7003A
:10723F0001992B030E0001995DD8B00ED000019972
:10724F0051010D0101E00EF324D96E0101010EF47D
:10725F0020DA6EDF50D8A4A1D7030E0001916F0082
:10726F000E00019B6FC9D000019B51010D00019CC5
:10727F000EF324D96E0001000EF420DA6EDF5000F9
:10728F0001A36FA9D05050D8B4B5D07F0E000161C3
:10729F006FF60E0001606F000150C062F0000163D5
:1072AF006B000E0001656F040E0001646FCDEC18CA
:1072BF00F0000160C093F0000161C094F0000194F0
:1072CF00519311D8B497D0060E0001A45DD8B09297
:1072DF00D00001A451010DF35000018725D96EF4A0
:1072EF005000018821DA6E2A0EDF6E0001A42BF602
:1072FF000E00018F6F7F0E906F00018F1F901F8FF9
:10730F004B902B0001935100018F270001945100E6
:10731F00019023840E00018F25F66E770E9021F7D2
:10732F006E0001A451010DF35000018725D96EF4B1
:10733F005000018821DA6E0800F5CFDFFF25D0500D
:10734F00500B0AD8A457D0060E0001A45DD8B05236
:10735F00D00001A451010DF35000018725D96EF41F
:10736F005000018821DA6E2A0EDF6E0001A42B0077
:10737F0001A451010DF35000018725D96EF450007F
:10738F00018821DA6E130EDF6E0001A42B0001A419
:10739F0051010DF35000018725D96EF4500001887B
:1073AF0021DA6E51C0DFFF14D00001968323D00085
:1073BF0001968B20D00001A451010DF350000187DD
:1073CF0025D96EF45000018821DA6E0001A3C0DFC9
:1073DF00FF0001A42B0FD00001A351E10AD8B4E4A0
:1073EF00D7040AD8B4E4D7160AD8B44CD7070AD8AA
:1073FF00B4A6D7E0D700019B2B030E00019B5DD8ED
:10740F00B012D000019B51010D00019C0EF324D945
:10741F006E0001000EF420DA6EDF50D8B404D007EE
:10742F000E0001A46520D7000E00016F6F500E00F3
:10743F00016E6F0001000E0001716F00019C0E00C4
:10744F0001706F000E0001736F030E0001726F2C3D
:10745F00EC18F083C0D9FF84C0DAFFDF504D6E0007
:10746F0001952B080E0001955DD8B004D0070E00D2
:10747F0001A46515D5020E0001A4651ED0010101FE
:10748F000E00016F6F0101E00E00016E6F000E0024
:10749F0001716F500E0001706F000E0001736F03CA
:1074AF000E0001726F2CEC18F087C0D9FF88C0DA7C
:1074BF00FF000196C0DFFF20D00101010E00016126
:1074CF006F0101E00E0001606F000E0001636F009D
:1074DF000E0001626F000E0001656F030E00016464
:1074EF006F20EC15F083C0D9FF84C0DAFF87C0E1AD
:1074FF00FF88C0E2FFDFCFE7FF00019151120000CC
:10750F000D0102030405060708090A1624000E0ED2
:10751F000E0E0E0E0E0E0B2F54180E0E0E41420EA7
:10752F000E0E235F550C0E0E0E4D4E0E0E0E175EE9
:10753F005619252627282B2C2D2E225D5730313218
:10754F0033343738393A3B5C583C3D3E3F40434437
:10755F004546475B5948494A4B4C4F505152535A35
:10756F002F3B3C3D3E3F40414243442E353A0000C5
:10757F000000000000004531301E00000000000038
:10758F000000272D2A1F2021220000232425263426
:10759F00141A09130A00000D0F181C3304151617BF
:1075AF000729650B11080C121D1B0619052B280E38
:1075BF0010363738E0E3F0E12CE2E62CE5F0E7E4B3
:1075CF002F3B3C3D3E3F404142434431353A000062
:1075DF00000000000000452E301E000000000000DB
:1075EF0000002738391F2021220000232425262DB3
:1075FF00343637131C0000090A06150F0412081839
:10760F000C2965070B17111633140D0E1B2B2805AC
:10761F00101A191DE0E3F0E12AE2E62CE5F0E7E4A9
:10762F00303B3C3D3E3F40414243442E893A0000AF
:10763F00000000000000452F321E00000000000077
:10764F000000272D391F2021220000232425263456
:10765F00141A08151700001C180C1213041607092A
:10766F000A29650B0D0E0F331D1B0619052B28114B
:10767F0010363738E0E3F0E12AE2E62CE5F0E7E4F4
:10768F00303B3C3D3E3F40414243442D893A000050
:10769F00000000000000452F321E00000000000017
:1076AF00000027342E1F2021220000232425262A04
:1076BF00141A08151700001C180C121304160709CA
:1076CF000A29650B0D0E0F331D1B0619052B2811EB
:1076DF0010363738E0E3F0E158E2E62CE5F0E7E466
:1076EF002F3B3C3D3E3F40414243442E353A000044
:1076FF000000000000004531301E000000000000B7
:10770F000000272D391F2021220000232425263495
:10771F00141A08151700001C180C12130416070969
:10772F000A29650B0D0E0F331D1B0619052B28118A
:10773F0010363738E0E3F0E12AE2E62CE5F0E7E433
:10774F00000000000000000000000000005500FBDA
:10775F0000675400005F606156005C5D5E57005922
:10776F005A5B28006200630000040C1808121CFA10
:10777F007F3B7FA67D0A1D0705D07D4900003B009A
:10778F00003C00003D00003E00003F0000400000B4
:10779F004100004200007F0000810000480000E02F
:1077AF004C003A0000000000000000000000000044
:1077BF00000000000000000000000000008000003A
:1077CF00470000E0E11DE01E000000000000000087
:1077DF00000000000000000000000000000000009A
:1077EF0000E027004600004C0000E01F00E02000F2
:1077FF00E02100E02200000000000000E02300E094
:10780F00E150E15200E0E14F530000E01400E01AB4
:10781F00004B0000E01500E0170000000000000022
:10782F00E04A00E05000520000E04F00E04D00E061
:10783F000400E016004E0000E00900E00A002900F5
:10784F00003900004A00005000005100004F0000B6
:10785F004D0000E01D00E01B00E00600E019009164
:10786F0000002B0000280000900000E15000E151C3
:10787F0000E14F00E14D000000000000000000009B
:10788F00000000E02A00000000000000E02C0000D3
:10789F0000000000000000000000000000000000D9
:1078AF0000000000000000000000000000000000C9
:1078BF0000000000000000000000000000000000B9
:1078CF000000000000000000000000B69AB5B4B33D
:1078DF0000002A31383F4604030201050000070E5D
:1078EF00151C23AE6993A4B200004D545BCD62000A
:1078FF000000000000000000000000000000000079
:10790F000000000000000000000000000000000068
:10791F00000000000000000000000000000000ACAC
:10792F00A9A6A2B00000307A3EC84CABA8A5A1AF63
:10793F0000000D141B2229ADAAA7A3B10000535AB2
:10794F0061CE68E600000000000000000000CA00E1
:10795F000000000000000000000000E70000000031
:10796F00000000000000CD0000000000000000003B
:10797F00000000CE08160C0F000039170A18CD03AF
:10798F0010190B120000241A0902C8CE2511262740
:10799F0000002E132028ECE600000000000000007D
:1079AF000000CA000000000000000000000000E717
:1079BF00CC000000000000000000CD00EDF1E6E774
:1079CF000000EAEB0000006A043A7F3C0000475DCC
:1079DF00505E4844011D812F000063604F4BC86CFF
:1079EF00C93D326B000049594A67ECE800000000BE
:1079FF00000000000000CB000000000000000000AD
:107A0F00000000E9CC000000000000000000CD00E5
:107A1F00EDF1E6E70000EAEB000000CE4E5C5255B8
:107A2F000000361E3B2B6D96565F515800002C05FB
:107A3F0021837ACE6457656600001F342D406ED3C4
:107A4F000000000000000000000000000000000027
:107A5F0000000000000000D4D7000000000000006C
:107A6F000000DE0000000000000000000000DD004C
:107A7F0000000000000000000000D1000000000026
:107A8F00000000000000000000DB0000000000000C
:107A9F000000E0D300000000000000000000000024
:107AAF000000000000000000000000D400000000F3
:107ABF00000000000000DE000000000000000000D9
:107ACF000000DF000000B300000000000000D20043
:107ADF000046D6D5000000D9D8DC00000000000019
:107AEF00000000DA000000E60000000000000000C7
:107AFF00000000000000000000000000000000E790
:107B0F000000000000000000000000000000000066
:107B1F0000000000000000393B0C24830000092105
:107B2F000A013C161A08192F000044020310C82B33
:107B3F003A1E0F1D00001118CDCE7AE6000000008E
:107B4F0000000000000000EE000000000000000038
:107B5F00000000E70000000000000000000000002F
:107B6F0000000000000000000000002513EC7F283B
:107B7F0000004F5150CC8E1F208136260000CA5D69
:107B8F009656906D6E1234270000575EEFF086E820
:107B9F0000000000000000000000000000000000D6
:107BAF0000000000000000E90000000000000000DD
:107BBF000000000000000000000000000000006452
:107BCF00595263670000040B2E2D3D5C604E5F65BC
:107BDF0000000517C92C3271745855660000406BB0
:107BEF006ACB6CE6000000000000000000000000FF
:107BFF000000000000000000000000E7000000008F
:107C0F00000000000000170000000000000000004E
:107C1F0000001D130B121983000018C821443A24C9
:107C2F0008101A1600000A0302CA09110C1E0F01D0
:107C3F0000007A3BCDCE3CE80000000000000000C1
:107C4F00000000000000000000000000000000E93C
:107C5F0000000000000000000000E600000000002F
:107C6F00000000000000E76ACB28262E0000250444
:107C7F002C321F6B2739813600002B052F40346CB7
:107C8F006D6E207F00002D3DECC9CC041111040E48
:107C9F0018041718040C000C11110C0E180C1718DF
:107CAF00181111180E18181718081111080E0C08B2
:107CBF001718080C00121111120E1812171812189B
:107CCF00000600000900000D000014000005010966
:107CDF0006A101050719E029E71500250175019592
:107CEF00088102950175088103950575010508192D
:107CFF0001290591029501750391039506750815E4
:107D0F000026FF000507190029FF8100C011112D62
:107D1F0000F300F400E13836003700E136E1372F89
:107D2F00003000E130E13234002E002D001E00380B
:107D3F00003200E1278700E136E137E138890000A2
:107D4F00000E001600170011000B0010001C00158C
:107D5F00001A0013000A001D00070005001B001B7E
:107D6F000E1B171B1C1B1A1A1C19000F00E0E1E356
:107D7F00E2E6E5E4E0E1E29190E5E4E0E1E3919011
:107D8F00E5E4E1E0E3E2E6E4E5E1E0E29190E4E559
:107D9F00E1E0E39190E4E52A034500730072006986
:107DAF00006C006C00650020004E0065007700201D
:107DBF00004B006500790062006F00610072006483
:107DCF000009022900010100A0320904000002038A
:107DDF000101000921110100012240000705810363
:107DEF000800010705010308000113062800001011
:107DFF00040628001E272104281E272105281E27D8
:107E0F002604281E27260528042D161328162D169E
:107E1F0013280612131C150C0A0B172C1F271E20D4
:107E2F00362C1F271E212C0816150C0F0F082C0C93
:107E3F0011063728091F2C002F0000300000E12FFA
:107E4F0000E13000E2E126E2E127380000380000CF
:107E5F00383838360000370000E135002F00003089
:107E6F0000002F00003000002F000030000038000D
:107E7F0000380000383838360000370000E1350090
:107E8F002F00003000001D2F001D30002F0000308C
:107E9F0000001D38003800001D3700360000370085
:107EAF0000E13500151210042800110C06122800ED
:107EBF0010171C13082817151211280016170C0677
:107ECF000E281B2327272128062800000000060D57
:107EDF0028000000060D10040628162800000000D8
:107EEF00160D28000000160D100406282F00003074
:107EFF0000002F00003000002F000030000038007D
:107F0F0000380000383838360000370000E13500FF
:107F1F000F28000006280000152800000F2D11283B
:107F2F00062D0628152D1628120909281A034500B3
:107F3F007300720069006C006C006500200049003E
:107F4F006E0063002E00181628000018162D072843
:107F5F0018162D06280D132800000D132D112808B3
:107F6F0016150C0F0F082C110C16160828150819CA
:107F7F00372C0007272800071E1F28071F21280757
:107F8F002023280721252810162800000417120E79
:107F9F00280A12120A280413130F281201000200D4
:107FAF00000008D80450F50100010200018B000009
:107FBF008A000088000035000012090928121128D4
:107FCF00000F080728190815372C0009262C00095F
:107FDF00202C0009212C0009222C0009232C000938
:107FEF00242C0009252C000E16170B04030904007E
:020000040020DA
:08000000FFFFFFFFFFFFFFFF00
:020000040030CA
:0E000000330E3F1EFF8181FF0FC00FE00F4047
:0200000400F00A
:080000000000000100040000F3
:00000001FF
